:100000000C9438000C9453000C9453000C9453003F
:100010000C9453000C9453000C9453000C94530014
:100020000C9453000C9453000C9453000C94530004
:100030000C9453000C94EA010C94FE010C94BE0144
:100040000C9453000C94D5010C9453000C94530061
:100050000C9453000C9453000C9453000C945300D4
:100060000C9453000C9453000C9453000C945300C4
:1000700011241FBECFEFD4E0DEBFCDBF11E0A0E062
:10008000B1E0E4E7F9E002C005900D92A030B107BD
:10009000D9F711E0A0E0B1E001C01D92AC31B10789
:1000A000E1F70C949A040C9400009FEF9ABB17BAE6
:1000B00081E484BB98BB8EEF85BBAE9880E48BBB9C
:1000C000089510BC8FEC89B986E880BD80E18AB9BB
:1000D000089580EA8FBD1EBC08950E9469000895AE
:1000E0008BB1992787FD90958827990F881F9927AD
:1000F00008951092130199278230910559F18330A8
:1001000091051CF4019749F080C08330910509F4F2
:1001100041C0049709F45BC078C010920A0181E0E5
:1001200080930D0180E88093010180E180930E01AE
:1001300080910601909107019093100180930F0127
:10014000809115019091160190930C0180930B0101
:100150008FE61DC081E080930A0182E080930D014B
:1001600080E88093010180E480930E018091150165
:10017000909116019093100180930F0180910601D8
:100180009091070190930C0180930B018FE3809372
:100190001901089510920A0183E080930D0180E215
:1001A0008093010180E480930E018091060190917B
:1001B00007019093100180930F0180911501909198
:1001C000160190930C0180930B018FE9E0CF81E041
:1001D00080930A0184E080930D0180E28093010105
:1001E00080E180930E01809115019091160190930A
:1001F000100180930F018091060190910701909367
:100200000C0180930B018FECC2CF1EBC10920E012B
:100210001092010110920D018FEFB9CF80910D0165
:1002200099278230910579F0833091051CF401976C
:1002300039F012C08330910549F0049751F00CC099
:10024000DF9ADC9810C0DE9ADF980DC0DD9ADE9848
:100250000AC0DC9ADD9807C01EBC10920E011092F5
:10026000010110920D011EBC8FEF809319011092B5
:100270000E011092010110920D0108959091130149
:1002800080911101980F90931301943618F480E037
:1002900090E0089594569093130181E090E00895C2
:1002A000089580910D01882309F466C080910A01A8
:1002B00040910F0150911001609102017091030172
:1002C00020910B0130910C01813081F5460F571FB1
:1002D0005093100140930F01261B370B30930C01F4
:1002E00020930B010E943E01892B91F080910F0118
:1002F0009091100101969093100180930F018091CD
:100300000B0190910C01019790930C0180930B01CC
:1003100020910F0130911001809106019091070109
:100320008217930748F50E940E010895260F371F84
:1003300030930C0120930B01461B570B5093100177
:1003400040930F010E943E01892B49F080910B01DF
:1003500090910C01019690930C0180930B012091D8
:100360000B0130910C0180910601909107018217D9
:10037000930710F40E940E01089508951F920F92A2
:100380000FB60F9211248F939F9389B39091190107
:1003900089238BBB81E080930401A8989F918F9162
:1003A0000F900FBE0F901F9018951F920F920FB6CF
:1003B0000F9211248F9383B382FF02C08B7F01C001
:1003C000846085BB81EB82BF8F910F900FBE0F9031
:1003D0001F9018951F920F920FB60F9211248F93B2
:1003E0009F9389B390910101892B8BBBA89A9F9110
:1003F0008F910F900FBE0F901F9018951F920F9224
:100400000FB60F9211248F939F9389B390910E0191
:10041000892B8BBB9F918F910F900FBE0F901F90D8
:100420001895982F80910901981711F410921A01CC
:1004300089B321E030E002C0220F331F9A95E2F722
:10044000922F909589238BBB0895382F883080F4A4
:1004500080910901381711F410921A0129B381E033
:1004600090E002C0880F991F3A95E2F7282B2BBB2A
:100470000895089599278730910509F466C088305A
:100480009105C4F48330910509F447C08430910587
:100490004CF48130910581F182309105B4F5892BBE
:1004A00041F108958530910509F444C006970CF098
:1004B00044C03DC08B30910509F462C08C30910579
:1004C00044F48930910509F450C00A970CF050C0EB
:1004D00044C08D30910509F463C08D3091050CF452
:1004E00057C08E30910509F463C00F9709F468C0B6
:1004F000089582E390E002C089E190E090930301C7
:100500008093020110921301089580E190E090938E
:1005100003018093020183E407C08CE090E0909394
:1005200003018093020182E38093130108958AE01E
:1005300090E0E4CF88E090E03DC087E090E09093C9
:100540000301809302018EE0EFCF86E090E090936C
:1005500003018093020189E1E7CF85E090E0909369
:1005600003018093020188E3DFCF85E090E0C6CFEE
:1005700084E090E0909303018093020187E3D4CF5D
:1005800084E090E0909303018093020181E1CCCF5D
:1005900083E090E0909303018093020185E5C4CF4E
:1005A00083E090E0909303018093020189E3BCCF44
:1005B00083E090E0909303018093020181E2B4CF45
:1005C00083E090E090930301809302018DE0ACCF33
:1005D00026B330E041E050E0822F9927817090707F
:1005E0008417950721F43F5F26953730A8F33830FC
:1005F00008F030E0832F880F8E5F80931B01832FDC
:100600000E943A02089510920D0110921401109266
:10061000080184E18093050110921A0110920901EA
:100620008FEF809319011092010110920E01109228
:10063000100110920F0110920C0110920B011092F8
:10064000130182E390E090930301809302011092E2
:1006500012011092110121E020930A01109204016D
:1006600085E58093000183EE9AED909318018093C5
:10067000170187E49BED90931601809315018BE998
:100680009FEF9093070180930601B79B04C02093CE
:100690001A010E94E802089508950E9455000E94E0
:1006A00003030E946D000E9461000895982F883016
:1006B00028F481E080931A01909309010895089528
:1006C0000E947000892BD1F18CB1282F2F70829558
:1006D0008F7099278330910521F1843091054CF476
:1006E00081309105B1F082309105BCF4892B69F01D
:1006F000089585309105D9F085309105A4F08630B4
:100700009105B9F00797B9F00895822F0E94110260
:100710000895822F0E9425020895822F0E943A0296
:10072000089581E001C082E00E947900089583E08D
:10073000FBCF84E0F9CF822F0E94560308950895DD
:100740009D9906C099B38FEF8BBB9D9BFECF9BBB42
:10075000089508958091050199278233910581F1CB
:10076000833391057CF48530910511F18630910534
:100770001CF4892BD9F008958A309105D9F00F9790
:10078000D9F008958634910509F1873491053CF438
:100790008C339105B9F081349105B1F008958B3413
:1007A0009105B1F08F359105A9F0089581E005C05C
:1007B000DA980895DB98089582E00E947900089500
:1007C00083E0FBCFD99A089584E0F7CFDA9A0895B1
:1007D000DB9A0895D9980895089580E09A99FDCFFD
:1007E0008F5F8A30D8F3089580E09A9BFDCF8F5FAA
:1007F0008A30D8F30895B79903C00E9460031FC0E0
:10080000809114018F5F8093140190911B018917CF
:10081000B0F010921401809108018F5F809308015D
:10082000843168F010920801809105018F5F8093F8
:100830000501843611F4109205010E94AA030E945A
:100840005101089580910D018823B1F010920401A7
:1008500080910F01909110019BBD8ABD80910B0189
:1008600090910C0199BD88BD80911701909118015C
:100870009DBD8CBD82E08EBD0895089580910D01CF
:10088000882341F080910401882321F480910401A0
:100890008130C1F71EBC109204010E94FB03B79B7C
:1008A00002C00E94E8020895089590E027E080FDCC
:1008B0009F5F8695215027FFFACF9170892F992746
:1008C000089580911A01882399F18091000188236D
:1008D00019F48FEF8093000180910001887B0E94C2
:1008E0005504582F409100013091090140FF0BC081
:1008F00029B381E090E002C0880F991F3A95E2F792
:10090000282B2BBB0CC029B381E090E002C0880FDC
:10091000991F3A95E2F7809528232BBB8BB3842F40
:10092000869580930001552319F08068809300011B
:1009300008950895CFEFD4E0DEBFCDBF0E944D03F0
:1009400080EE89BF78940E94ED03C0E00E94A0036E
:10095000C13029F40E94ED03C0E0AE9A04C00E94A9
:10096000F403C1E0AE980E9422040E943E040E945B
:040970006104ECCF63
:00000001FF
